:020000040000FA
:0600000000008A01B02996
:08000800F000030E8301F1007A
:100010008B1029108513721D0F2876207211291D4F
:1000200045282910A10A0A302106031D2A28A1010A
:10003000A20A0A302206031D2A28A201A30A0A30B6
:100040002306031D2A28A301A40A0A302406031D3F
:100050002A28A40121082E06031D622822082F0643
:10006000031D622823083006031D62282408310678
:10007000031D6228A91C41282914851772150B122B
:100080006228762029148517622800000930A10310
:10009000A11F5728A100A203A21F5728A200A30353
:1000A000A31F5728A300A403A41F5728A4002108B6
:1000B000220423042404031D6228291485177215C1
:1000C000A9180B12710E8300F00E700E0900820742
:1000D0003F3406345B344F3466346D347D3407343A
:1000E0007F346F340034403450341834B208031D68
:1000F00008008B100B16721129108513291D8528F5
:10010000A101A201A301A40108002E08A1002F084B
:10011000A2003008A3003108A40008000C30A90692
:1001200008000230A9068B100B1608002108672072
:10013000A50022086720A60023086720A70024083E
:100140006720A800F21C0800B208031D08000A304E
:100150006720A408031D0800A800A308031D0800C9
:10016000A700A2080319A600080005088039850029
:100170001030AA0C0318AA002A18250DAA18260D5B
:100180002A19270DAA19280D2A1A290D7218FF3AC3
:100190008600050880392A04850000000000000060
:1001A000051BAB042A09051FAB052A1C0800A00B80
:1001B00008000530A0002C082B062B05AD002B08ED
:1001C000AC00F21508000B120B12B208031DF12847
:1001D0000B30A400A300A200A101B20A21308400C8
:1001E00008000408243A0319F828840A800108004A
:1001F0002108AE002208AF002308B0002408B10097
:10020000A101A201A301A401B2019B218B100B1635
:100210000800B20803190800800A00080A3A031906
:10022000800108001030B20024210C1D15290C118A
:10023000B520F21D1529F2112D1A2421AD1D152905
:10024000B2015521762008000830B20C0318B20024
:1002500032184B29B2184129321938292F29F210A6
:1002600072120D30A4000030A300A200A100962855
:10027000F21072160C30A4000030A300A200A100FE
:100280009628F21472120D30A4000A30A300A200C6
:100290000030A1009628F21472160C30A4000A3027
:1002A000A300A2000030A1009628000083120317CB
:1002B0008D0172085E21831203130800000083126F
:1002C00003130D12831203178C00831603178C136C
:1002D0000C158B138B1B692955308D00AA308D00AE
:1002E0008C140C118B17831203130D1E75298312A6
:1002F000031708000000831203178D0083160317ED
:100300008C130C14831203170C08831203130800B8
:1003100003017A211239F2000800000001307A212D
:10032000B10002307A21B00003307A21AF000430EE
:100330007A21AE00080000000130831203178D00FF
:10034000831203133108A9213008A9212F08A921FC
:100350002E085E21831203178D0A831203130800EF
:1003600083018601831670308F00003081009B016D
:1003700001308600603085008312FF30860008302F
:1003800085008020A9010030AE00AF00B000B100B0
:100390002915A911FF30AB00AC000530A0000430D6
:1003A00092000B309700D030950007309600013056
:1003B000900088218D2172141030AA00051B122193
:1003C000B2018316721A011783120B168B170C19C0
:1003D000EA21E7290C119620B520F21D0800F21140
:1003E0002D188E20AD1876202D199120AD19E320FF
:0603F0002D1A092108008E
:02400E00703F01
:02401000FC3F73
:084202000000000000000000B4
:1042100063006F0075006E0074006500720032006C
:0E4220003000300039002E00610073006D0088
:00000001FF
